:020000040000FA
:020000005B2B78
:080008009600030E97000A08A0
:1000100098000A108A1083123F309C1A1D08810232
:1000200019089A071A0C95003F39951A403C2E2062
:10003000151B103C95000608F039150486009C0B32
:1000400026281B089900941420309C000B111808D6
:100050008A00170E8300960E160E090082070834D8
:1000600008340934093409340A340A340A340B34A4
:100070000B340B340C340C340C340C340D340D3480
:100080000D340D340E340E340E340E340E340E3462
:100090000F340F340F340F340F340F340F340F3448
:1000A0008B018316F03086058B1283165730810042
:1000B00083128B1308000C3037239D0008309B00FF
:1000C00083165830810083128B168B170800941CFE
:1000D00067281B08031C173C9B009410080082072C
:1000E0000034023406340D341B3436345134861B4C
:1000F000073E8207963418340C3406340334023435
:100100000134B4341E34103408340434033402345B
:100110009F011F08383E840000308A001F08972086
:1001200080009F0A1F080E3A031D8928382982077C
:100130008A34A434A4349E34A434423460344E341B
:100140004F34203447345034533420348F009E08C9
:10015000031DDD2800308A001F08C0200F06031D84
:1001600038299F0A2C300F06031D08003230840006
:1001700030308000840A0408383A031DB8282F293B
:100180000739820724344734503452344D344334D1
:100190002C3482070034003401340634013407342F
:1001A0000134033403348207003400340034013452
:1001B000073408340F34103413340F082C3A031961
:1001C0002F290F082A3A0319382900308A001E08FF
:1001D000C9201F06031908001E08063C031CFF283F
:1001E0000F082E3A0319080000308A001E08D32099
:1001F0001F07223E84000F0880009F0A08000F0896
:100200002E3A0319162900308A001E08D320223EF8
:100210008400840A000884038000840A840A000899
:1002200084038000840A0F088000080000308A00E0
:100230001E08C9209F00080006308E0000308A008A
:100240000E086F200D02031828298E03031D1E2996
:100250000E08210203182E290E08A10008009F0194
:100260009E0A1E08093A031D08003B21CC21CD003F
:100270009F019E010800223084000008413A273087
:1002800003196030A001BF00840A9F01000D9E0089
:10029000153084071E081E3960388000EC30840752
:1002A0009F0A1F08063A031D4629063037239F0080
:1002B000C0301F1CBA069F1CB9061F1DB806A9191D
:1002C000BB062A18BC06B118BD0607303723BE008E
:1002D0000310BE0DE0382B30A7211C3EC0002D308E
:1002E000A7211C3EC1002F30A7211C3EC200323086
:1002F000AA218D001C210D08C400C30101308A0011
:100300000A30C30AC40203188129C3034407C02169
:10031000C4006C30C3073530840000080F39203E1C
:10032000C4073630A7211C3EC5002D080F393C30CC
:100330000319C1072B080F39031D08005030C007EF
:10034000BC1B08000A30C007BC173C13080084001F
:100350009E01B129840001308A000008BB219E0063
:10036000840A01308A000008C0219E07840A000820
:100370000F391E0708000339820700346434C8347B
:100380000F39820700340A3414341E3428343234CE
:100390003C34463450345A343F08603A031DFF342D
:1003A0003230AA21073C0318FF344508E43E92008E
:1003B0000310920C35080F39930032300319E329EA
:1003C00092079303DE29120808004E0A031D003429
:1003D0004C0A031900344D08013E03190034FF3E56
:1003E0004C02031C003C9300861B1D3C861F133CE3
:1003F000031800341308861B973C861FA13C031C7E
:1004000000340134F530CE004D08013E03190800D8
:10041000FF3ECC0008000515582238308400000843
:100420006522840A04083F3A031D0F2A003037234F
:100430008E000E08372300380319212A65228E0A00
:10044000192A00086522840A0408463A031D212A55
:100450000830372365220930372365228C0B3E2A6A
:10046000033037238C00043037238E000E083723E7
:10047000003803193E2A65228E0A362A7A2205118F
:100480000800910D110C672011091F39031D080088
:100490000310412A00304F2AFF304F2A7E308F0050
:1004A000083090008F0C41229101900B522A0800D5
:1004B0000130861B0A3037238D005B204E228D0BC6
:1004C0005E2AFF309200930008008F0008309000F1
:1004D0000F0C0130031893060310920C930C031CAD
:1004E000752A08309306843092068F0C4122900BB7
:1004F000682A0800FF30930612068D001308652253
:100500000D0865224E224E22542008009100000062
:10051000910B882A08008316051685118312851110
:1005200008008F000A30900003108511031C851508
:10053000A930862203148F0C900B952A08000F1007
:10054000051E003409309000383086220310051E45
:1005500003148F0CA93086220000900BA62A0F08E6
:10056000051AB02A0F1408009F220F1CB42A080095
:1005700083168510051083120130C800C700FF30B4
:10058000CA00A000C900CC00CE00A101CB01080028
:10059000061EC90146080102C607031C0800031015
:1005A000861E0314CB0DC70B08002630C700C90AEE
:1005B0000319C903061EC901A00A0319A003CE0A24
:1005C0000319CE03C80B08000A30C800CA0A031971
:1005D000CA030800C822C9080319F52A05303723C1
:1005E0004902031CF52A0510F62A05142008043CCC
:1005F0000318012B85103F08603A27300319BF000C
:10060000092B3F08603A03190E2B471A8514471E21
:1006100085104B08FE3A031D362B302B85144B08F2
:10062000FE3A031D152BFF30CA00061B1D2BE521CA
:10063000003803191D2BFF30CA0000308A00210842
:100640007720061F282B861F0230861B0B3037238E
:100650004A02031C362B053037234902031C362B74
:100660000222CA01A1013821CB01013400343F39F3
:100670008900831608148312080808003F3989008E
:1006800083168B13081555308900AA308900881409
:1006900008118B1788184A2B83120800851405143B
:1006A0005523851005105523080000008D0B552B90
:1006B0009D0B552B08008B2288205020B8228316D2
:1006C00005118312051155234E234E234E2301306D
:1006D0008C009F220F1C722B8D001B3A0319772B65
:1006E0000D08A620EA220038031D0B22692BB42234
:1006F0008D001B3A0319772B0D08443A03198D2BF3
:100700000D08553A0319972B0D08563A03199F2BDC
:100710000D08543A0319C12B692B8D01B4228800AE
:100720000D083E238D0A0D1F8E2BB822692B8D01DB
:100730000D08372391228D0A0D1F982B692B8D01EF
:1007400003308A000D08AB2300380319AA2B91222D
:100750008D0AA02B692B8207543469346E347934A6
:100760005434723461346B3420343434533436347A
:100770004734473453342034563430342E343934EB
:100780000034B4228D00303A0319CF2B0D08313AD2
:100790000319D92B0D084D3A0319E32B692B851446
:1007A000051005155B204C22051ED32B0511542086
:1007B0005B2B8510051405155B207F304F224C22E2
:1007C000051EDF2BD62B8514051405155B204A2248
:0607D000051EE72BD62BED
:02400E00F23F7F
:104200000D0028000C0003001E0003000000000049
:104210003E002F000A0003003F009C009E00860025
:104220008200980098006000A4008A009800820034
:10423000B200400061000300F000000020002000F8
:104240003400530036004700470053002000200090
:0C42500047006100790061006E00000072
:00000001FF
